:020000040800F2
:1000000000040020E1010008CD0C0008CD0C000820
:10001000CD0C0008CD0C0008CD0C0008CD0C00085C
:10002000CD0C0008CD0C0008CD0C0008012B0008F9
:10003000CD0C0008CD0C0008CD0C0008CD0C00083C
:10004000CD0C0008CD0C0008CD0C0008CD0C00082C
:10005000CD0C0008CD0C0008CD0C0008CD0C00081C
:10006000CD0C0008CD0C0008CD0C0008CD0C00080C
:10007000CD0C0008CD0C0008CD0C0008CD0C0008FC
:10008000CD0C0008CD0C0008CD0C0008CD0C0008EC
:10009000CD0C0008CD0C0008CD0C0008CD0C0008DC
:1000A000CD0C0008CD0C0008CD0C0008CD0C0008CC
:1000B00019240008CD0C0008CD0C0008CD0C000858
:1000C000CD0C0008CD0C0008CD0C0008CD0C0008AC
:1000D000CD0C0008CD0C0008CD0C0008CD0C00089C
:1000E000CD0C0008CD0C0008CD0C0008CD0C00088C
:1000F000CD0C0008CD0C0008CD0C0008CD0C00087C
:10010000CD0C0008CD0C0008CD0C0008CD0C00086B
:10011000CD0C0008CD0C0008CD0C0008CD0C00085B
:10012000CD0C0008CD0C0008CD0C0008CD0C00084B
:10013000CD0C0008CD0C0008CD0C0008CD0C00083B
:10014000CD0C0008CD0C0008CD0C0008B92100082A
:10015000CD0C0008CD0C0008CD0C0008CD0C00081B
:10016000CD0C0008CD0C0008CD0C0008CD0C00080B
:10017000CD0C0008CD0C0008CD0C0008CD0C0008FB
:10018000CD0C0008CD0C0008CD0C0008CD0C0008EB
:10019000CD0C0008CD0C0008CD0C0008CD0C0008DB
:1001A000CD0C0008CD0C0008CD0C0008CD0C0008CB
:1001B000CD0C0008CD0C0008CD0C0008CD0C0008BB
:1001C000CD0C0008CD0C0008CD0C0008CD0C0008AB
:1001D000CD0C0008CD0C0008CD0C0008CD0C00089B
:1001E00072B6374880F3098836484EF60851CEF289
:1001F0000001086040F20000CCF200004EF63471BD
:10020000CEF200010860BFF34F8FBFF36F8F40F253
:100210000000C0F2F0004EF68851CEF200010860F6
:10022000BFF34F8FBFF36F8F4FF00000E1EE100A66
:100230004EF63C71CEF200010860062080F314886F
:10024000BFF36F8F00F024FD02F026F94FF0553018
:100250001D491E4A91423CBF41F8040BFAE71C4974
:10026000174A91423CBF41F8040BFAE719491A4A70
:100270001A4B9A423EBF51F8040B42F8040BF8E7C0
:1002800000201749174A91423CBF41F8040BFAE796
:1002900000F002FD02F002F9134C144DAC4203DAF7
:1002A00054F8041B8847F9E700F03EF8104C114D54
:1002B000AC4203DA54F8041B8847F9E700F0EABCC3
:1002C00000080020000000080000002000040020BA
:1002D00000040020A835000800080020280800209D
:1002E00028080020301A0020E0010008E001000882
:1002F000E0010008E00100082DE9F04F2DED108A23
:10030000C1F80CD0C3689D46BDEC108ABDE8F08FE3
:10031000002383F311882846A047002000F0DAFE6E
:1003200000F074FE00DFFEE738B5174B7D22002495
:100330001A700F225C709C70DC701C715C719C7177
:10034000DC711C725C729A72DC7202F0FBFA0F4B69
:10035000984217D00133984241F2883412BF0025E9
:1003600000240125002002F0F3FA0DB100F052F84C
:1003700000F062FC00F022FB204600F091F800F053
:1003800049F8F9E72546EDE728080020010007B005
:1003900008B500F0B5FAA0F120035842584108BD55
:1003A00007B5054B02211B88ADF8043001A800F009
:1003B000F5FA03B05DF804FB7832000810B5114877
:1003C000C3680BB100F04EFD0F4C104A0D480023DE
:1003D0004FF47A7100F00AFD236813B12368013BE2
:1003E0002360636813B16368013B6360084B1B784B
:1003F00033B9636823B9022000F0CEFB3223636077
:1004000010BD00BF340800204C0D0020BD030008C3
:100410004808002038B51B4C2368013330D01A4DF2
:100420001A4B2A689A422BD9194B9B6803F1006337
:1004300003F580339A4223D2002000F0D9FA154BFD
:100440000220187000F096FB134B1A6C00221A64FD
:10045000596C5A64596941F0800159615A611969AE
:1004600041F0005119611A6172B60C4B1C6023688F
:100470002A68202181F311889D4683F3088810475C
:1004800038BD00BF0000010804000108FFFF00089C
:1004900028080020480800200038024008ED00E04D
:1004A0002DE9F04FB34B8246B3489C680022C260EE
:1004B0008FB0202282F31188C26800930AB100F045
:1004C000D1FC0023AD4AAC484FF47A7100F08EFCA9
:1004D000002383F31188DFF8C0B2BAF1000F01D016
:1004E000CBF800A0A64FCBF8043000253B702E4679
:1004F0004FF0FF38012000F03DFBBAF1000F00F093
:10050000C181DBF80030002B40F0BC810FB0BDE8AA
:10051000F08F0220FFF73CFF002840F0AF81994B9D
:100520001B88ADF82430022109A800F037FAE1E772
:100530004FF47A7000F0E4F9031E0193EFDB022020
:10054000FFF726FF81460028E9D0019B581E0428AA
:10055000E5D8DFE800F00310131619000EA80523F4
:1005600040F8143D042100F019FA4D4600F05AFB02
:10057000FFF716FF7FE104217E48F4E7042182485B
:10058000F1E704218148EEE71C25284600F032FA05
:1005900004350990042109A800F000FA2C2DF4D1AB
:1005A000E3E7002EBBD0002DB9D00220FFF7F0FE0C
:1005B000064610B901252E46B1E7012000F018FAD1
:1005C0000220387000F0D6FA00255FFA85F9484617
:1005D00000F026FA0135044618B1484600F030FA1A
:1005E000F3E7012302203B7000F0B2FA009B9B6806
:1005F0009C4207D2204600F0FDF9013040F04081D6
:100600000434F3E700243C70CBF804403546ADE7F2
:10061000002E84D0002D82D00220387000F0AAFA7B
:10062000322000F06DF9051EC4DB15F00306C1D1C0
:10063000009A926863199342BCD8B5F5807FB9D807
:10064000DFF84C91AE420CDA4FF47A7000F058F9B2
:100650000390039B002BADDB039B06F809300136AA
:10066000F0E7C820FFF794FE06460028A2D02CB978
:10067000474B4FF0FF32D3F800801A60444B25F00F
:1006800003052544A3EB0409AC42BFD059F804107C
:10069000204600F0B5F9204600F0ACF959F80430D6
:1006A000984240F0ED800434EEE70220FFF770FE40
:1006B00000283FF434AF4FF0000AD146009B9B68FE
:1006C0009A4537D2BAF1000F17D1B8F1FF3F14D0D5
:1006D000CDF824802F494B68A3B1002209A8135CF0
:1006E00083EA0903DBB2013251F82330042A83EA9A
:1006F0001929F4D10AF1040AE0E7504600F07AF92A
:100700000990E7E71A46082012F0010F4FEA52025B
:100710001FBF82F06D4282F4380282F4034282F0FD
:1007200020020138F0D141F823200133B3F5807F56
:10073000E8D1D2E70EA8042140F8289D00F02EF958
:1007400014E70EA8002340F8143D642100F002F9DC
:1007500000287FF4E4AE0220FFF71AFE00283FF4E1
:10076000DEAE099800F07EF90EAB43F8240D0421AB
:100770001846E3E72808002034080020BD030008DD
:10078000480800207A3200082C0800203008002099
:100790004C0800204C0900204C0D00200EA800231E
:1007A00040F8143D642100F0D5F800287FF4B7AE7E
:1007B0000220FFF7EDFD00283FF4B1AE099800F0EC
:1007C0005FF90EAB43F8200DD1E70220FFF7E0FD03
:1007D00000283FF4A4AE00F059F90EAB43F81C0D0D
:1007E000C5E70220FFF7D4FD00283FF498AE09A921
:1007F000142000F051F981460EA8042140F8189DFC
:1008000000F0CCF8494609A898E74FF47A70FFF752
:10081000BFFD00283FF483AEB8F1FF3F05D1FFF7DD
:10082000BFFD354800F05CFC70E64146002000F05A
:10083000E7F8002000F0DEF88045F0D02F4B6FE69F
:100840000EA8002340F8143D642100F083F800282E
:100850007FF465AE0220FFF79BFD00283FF45FAEFA
:10086000FFF79EFD41F2883000F03AFC099800F055
:100870000DFA00F0D7F94FF0000A3BE6064675E6A0
:100880003546DBE7002000F03BF80390039B002B8C
:10089000FFF633AE012000F05BF9039B213B122BE6
:1008A0003FF628AE01A252F823F000BF130500085E
:1008B00031050008A3050008F5040008F504000848
:1008C000F504000811060008F5040008AB0600084E
:1008D000430700089D070008CB070008F50400083F
:1008E000E3070008F50400080B0800086D05000880
:1008F000F504000841080008A08601007C320008C9
:1009000037B5114A12780132D2B20024012A0346C7
:100910008DF8074011D80D480268D5694FF47A72F6
:1009200053430DF107010122A847012805D1084BC7
:100930009DF807001C7003B030BD4FF4FA7000F052
:10094000CFFB4FF0FF30F6E700080020D810002062
:10095000580D002038B50E4B1A780132D2B2012A58
:1009600005460ED80B480368DC694FF47A734B4395
:1009700004222946A047042803D1074B0020187001
:1009800038BD4FF4FA7000F0ABFB4FF0FF3038BDCC
:1009900000080020D8100020580D002030B4054C6D
:1009A00023689D69044B0A46AC460146204630BC8C
:1009B000604700BFD8100020A086010070B501F08C
:1009C000FDFE094C094E20700025306823788342D3
:1009D00008D901F0EDFE336805440133B5F5803FD9
:1009E0003360F2D370BD00BF590D0020540D0020BC
:1009F00001F094BF00F1006000F58030006870479E
:100A000007B502AB00F1006043F8041D042219464B
:100A100000F5803001F010FF03B05DF804FB00002A
:100A2000054B1A68054B1B781344834202D91044C6
:100A300001F0BEBE00207047540D0020590D00206B
:100A400038B5074D04462868204401F0B9FE28B99E
:100A500028682044BDE8384001F0CABE38BD00BF58
:100A6000540D002010F0030308D1B0F5007F05D825
:100A700000F10050A0F50840006870470020704762
:100A8000014BC058704700BF107AFF1F014B186818
:100A9000704700BF002004E070B52A4B1C68C4F307
:100AA0000B03240C63B140F21342934231D040F265
:100AB000194293422FD040F2214293422DD1032379
:100AC000214A0C2505FB03235D6893F9082042F2B7
:100AD00001039C4224D0B4F5805F23D041F201038E
:100AE0009C4221D041F203039C421FD041F20703F4
:100AF0009C4208BF3122441E0C44013D0B46A342D8
:100B00001ED215F9016F581C96B1034600F8016C0E
:100B1000F5E70123D4E70223D2E73F220B4DD6E7C6
:100B20003322E3E74122E1E75A22E4E75922E2E7F0
:100B30002C2584421D7001D9981C5A70401A70BD32
:100B40001846FBE7002004E08C32000880320008E1
:100B5000022804D1054B4FF000729A6170470128BA
:100B6000FCD14FF08042024BF7E700BF0004024087
:100B700000000240022804D1054B4FF400729A6134
:100B800070470128FCD14FF48042024BF7E700BFC9
:100B90000004024000000240022805D1064A5369C1
:100BA00083F40073536170470128FCD1034A5369F1
:100BB00083F48043F6E700BF0004024000000240D7
:100BC00010B50023934203D0CC5CC4540133F9E741
:100BD00010BD000030B5441E14F9010F0B4660B182
:100BE00093F90050854201F1010106D11AB993F938
:100BF0000020801A30BD013AEEE7002AF7D11046F6
:100C000030BD000002460346981A13F9011B002963
:100C1000FAD1704702440346934202D003F8011B05
:100C2000FAE77047024B1A78024B1A70704700BF00
:100C3000580D00200008002038B5104D104C2846F3
:100C400000F010FB2146284600F038FB23680D48D1
:100C50005A6DD2F8043843F00203C2F8043800F0A9
:100C60003FFA0949206800F041FC23685A6DD2F828
:100C7000043823F00203C2F8043838BDD81000202D
:100C80008834000840420F00D43400087047000048
:100C900070470000FEE70000084A094B09498B42F3
:100CA00004D3094A0021934205D3704752F8040F38
:100CB00043F8040BF3E743F8041BF4E7CC350008D2
:100CC000301A0020301A0020301A00201EF0040FC5
:100CD0000CBFEFF30880EFF309808169004A1047E9
:100CE000E90C000870470000204B02681A60204B96
:100CF00042681A601F4B82681A601F4BC2681A60F4
:100D00001E4B02691A601E4B42691A601D4B8269B4
:100D10001A601D4BC2691A601C4B1D491A681D4B95
:100D20001A601A68120A0A701A681B4B1A701B4B59
:100D30001A681B4B1A601B4B1A681B4B1A601B4B23
:100D40001A681B4B1A601B4B1A681B4B1A601B4B13
:100D50001A681B4B1A601B4B5A6A1B4B1A601B4BC1
:100D60001B68DB0701D500BEFEE7FEE78C0D002007
:100D7000900D0020980D00209C0D0020940D002067
:100D8000800D0020840D0020880D002028ED00E05B
:100D9000640D0020680D0020780D00202CED00E08F
:100DA000700D002030ED00E06C0D00203CED00E007
:100DB0005C0D002034ED00E0740D002038ED00E003
:100DC000600D002000ED00E07C0D0020F0ED00E063
:100DD000054B03F114025A619A614FF0FF32DA6158
:100DE00000221A62704700BFA00D0020F8B5036111
:100DF0004FF08043C2605C6A194B1A46022952F8D0
:100E0000145F38BF0221954206461F460AD1586139
:100E100098611C620560456081600819BDE8F84072
:100E200000F042BB186AAB68241A0C1902D3E41A0A
:100E30002D6804E09C4202D2204400F043FBAB68E2
:100E40009C42F4D86B68736035601E606E60B4605D
:100E5000A9684FF0FF33091BA960FB61F8BD00BF13
:100E6000A00D002010B41B4C234653F8141F8142E0
:100E700010D0416802680A60026851609A424FF0DF
:100E80000001C16003D0936881680B4493605DF8F2
:100E9000044B70470A68626100209A425360C86040
:100EA00003D15DF8044B00F007BB936888680344E6
:100EB00093604FF08042506A226A821A9342E6D9C8
:100EC0009B1A022B2CBFC01802305DF8044B00F0B7
:100ED000F9BA00BFA00D0020024B00221B605B602E
:100EE0009A607047A00D0020002303748268054BB0
:100EF0001B6899689142FBD25A6803604260106097
:100F000058607047A00D002008B5202383F3118896
:100F1000037C032B05D0042B0DD02BB983F3118850
:100F200008BD436900221A604FF0FF334361FFF7A9
:100F3000DBFF0023F2E790E80C001A6002685360C0
:100F4000F2E70000002303748268054B1B68996870
:100F50009142FBD85A680360426010605860704745
:100F6000A00D0020054B19690874186802681A6002
:100F70005360186101230374FFF7BEB9A00D002070
:100F800030B54B1C87B005460A4C10D023690A4A7D
:100F900001A8FFF72BFF2846FFF7E4FF049B13B1DE
:100FA00001A8FFF75FFF2369586907B030BDFFF75D
:100FB000D9FFF8E7A00D0020090F000838B50C4D47
:100FC00041612B6981689A689142044603D8BDE863
:100FD0003840FFF789BF1846FFF786FF01232C61D1
:100FE000014623742046BDE83840FFF785B900BFAD
:100FF000A00D0020044B1A681B6990689B689842FA
:1010000094BF002001207047A00D002010B5084CAF
:10101000236820691A6822605460012223611A74CF
:10102000FFF790FF01462069BDE81040FFF764B963
:10103000A00D002008B5FFF7DDFF18B1BDE808409E
:10104000FFF7E4BF08BD00008260022202740022A4
:1010500042748261704700008368A3F1840243F800
:10106000142C026943F8442C426943F8402C084A86
:1010700043F8242CC26843F8182C022203F8102CE1
:10108000002203F80F2C43F8082CA3F1200070472E
:101090001103000808B5FFF7DFFFBDE80840FFF7C0
:1010A00023BF000010B5202383F31188FFF7D4FF7E
:1010B00000210446FFF782FF002383F311882046B6
:1010C00010BD0000024B1B6958610F20FFF74ABF9B
:1010D000A00D0020202383F31188FFF7F3BF000049
:1010E00008B50146202383F311880820FFF748FF45
:1010F000002383F3118808BD10B5054C23690360F4
:1011000058610320FFF72EFF2369586910BD00BF07
:10111000A00D002003682BB100220260596118461F
:10112000FFF7E2BE7047000049B1064B42681B69F9
:1011300018605A60136043600420FFF721BF4FF02E
:10114000FF307047A00D00200368984206D01A684F
:101150000260506059611846FFF7C6BE7047000034
:1011600038B504460D462068844200D138BD036876
:1011700023605C604561FFF7B7FEF4E713B5446B8D
:10118000D4F88C341A681178042916D1217A0229EE
:1011900013D11979128901238B4013420DD101A972
:1011A00004F1440001F008FE024630B1D4F88C444A
:1011B000019B2179206800F0E5F902B010BD000024
:1011C0000C3001F077BD00004FF0FF330C3001F020
:1011D00071BD0000443001F05BBE00004FF0FF33F2
:1011E000443001F055BE00000C3001F045BD000058
:1011F0004FF0FF310C3001F03FBD0000443001F0F2
:1012000027BE00004FF0FF32443001F021BE000045
:10121000D0F88C2438B5136819780429054601D014
:10122000012038BD017A0229FAD112795C890120A6
:1012300090400440F4D105F10C0001F0D7FC0246C7
:101240000028EDD0D5F88C544FF480732868697964
:1012500000F086F9204638BD406BFFF7D9BF00008B
:10126000704700007FB50346114A43F8042B01255F
:10127000436002260F4B057204460290019300F171
:101280007C02294600964FF480730C3001F08AFCF2
:10129000094B0193029400964FF4807304F5217278
:1012A000294604F1440001F063FD04B070BD00BFA5
:1012B000DC320008591200087D1100080B6820225A
:1012C00082F311880A7903EB820290614A7909322C
:1012D00043F822008A7912B103EB8203986102235A
:1012E0000372C0F88C14002383F311887047000048
:1012F00038B5044601250221043001F0DDFB04F17C
:101300000C0025756FF00101FFF72AFF84F84C509F
:1013100004F144006FF00101BDE83840FFF720BF41
:1013200010B501210446043001F0C6FB00232375EB
:1013300084F84C3010BD000038B5044600250C3050
:1013400001F048FC04F14400257501F029FD201D41
:1013500084F84C50012101F0AFFB2046BDE8384035
:10136000FFF756BF90F8443003F06003202B19D1EB
:1013700090F84520212A0AD0222A4FF000030ED0EF
:10138000202A0FD1084A82630722C26304E0064B79
:1013900083630723C36300230364012070478363CF
:1013A000C363F9E70020704701080020D0F88C34AF
:1013B00037B51A681178042904461AD1017A02292E
:1013C00017D11979128901238B40134211D100F1F1
:1013D0004405284601F0BAFD58B101A9284601F09C
:1013E000EBFCD4F88C44019B21790246206800F084
:1013F000C9F803B030BD000000EB8103F7B59C696C
:1014000005460E46F4B1202383F3118805EB8607C9
:10141000201D082101F050FBFB685B691B68443408
:1014200013B1204601F0D6FC01A9204601F0C4FC0E
:10143000024648B1019B3146284600F0A3F800233C
:1014400083F3118803B0F0BDFB685A691268002A63
:10145000F5D01B8A013B1340F1D105F14402EAE7C4
:10146000093110B550F82140CCB1202383F3118805
:101470000421601801F020FBD4F88C241368527901
:1014800003EB820304F10C00DB689B69596801F0EF
:10149000B7FB2046FFF7BCFE002383F3118810BD85
:1014A0007047000000F0CCBF4FF08043002258632B
:1014B0001A610222DA6070474FF080430022DA603E
:1014C000704700004FF080435863704700F09CBBAA
:1014D0000123037000234360C36183620362C3621C
:1014E00043620363038143817047000038B50446BB
:1014F000202383F3118800254160C56005614561A3
:10150000856100F093FB0223237085F3118838BDB9
:1015100070B500EB810305465069DA600E4614464B
:1015200018B110220021FFF775FBA06918B1102235
:101530000021FFF76FFB31462846BDE8704000F000
:101540004DBC0000028902F001020281428902F0D2
:1015500001024281002202614261826100F0D2BC3C
:10156000F0B400EB81044789E4680125A4698D404B
:101570003D43458123600023A2606360F0BC00F01E
:10158000EDBC0000F0B400EB81040789E46801259C
:1015900064698D403D43058123600023A260636040
:1015A000F0BC00F06BBD000070B5022300250446BE
:1015B0000370A0F84C5080F84E5080F84F500581D1
:1015C0004581C56005614561856180F8345000F052
:1015D000A3FB63681B6823B129462046BDE8704021
:1015E000184770BD436802781B6880F850200522B8
:1015F00002700BB10421184770470000436890F84F
:1016000050201B6802700BB105211847704700007D
:1016100070B50023044680F8343000F1440200F035
:1016200093FC63689B685BBB94F8445015F06006BC
:1016300014D194F8453005F07F0545EA0325B5F54A
:10164000407F00F0A58059D8022D00F0F1803FD8EE
:10165000002D00F08780012D00F0E480002120465D
:1016600000F0BCFE0021204600F0AEFE63681B685F
:1016700013B1062120469847062384F8343070BD04
:10168000204698470028CFD094F84B2094F84A3051
:1016900043EA0223E26B934238BFE36394F9443098
:1016A000E56B002B4FF0200380F20181002D00F04C
:1016B000F080012284F8342083F311880021E36B49
:1016C000A26B2046FFF75EFF002383F3118870BDF5
:1016D000B5F5807F4DD0B5F5817FBFD194F8463008
:1016E000002BBBD194F8483013F00F0126D01A0616
:1016F000204640F1B78000F085FE1FE0B5F5C06FD1
:1017000050D020D840F202339D4200F0AE80B5F5B3
:10171000A06FA3D1B4F84430B3F5A06F0ED194F804
:10172000463084F84E30204600F04CFB63681B685E
:1017300013B1012120469847032323700023A3639C
:10174000E3632364A0E7B5F5106F41D040F6024390
:101750009D4267D0B5F5006F80D104F14F03A363BC
:10176000012333E004F14C03A3630223E363256404
:101770008AE794F84630012B7FF470AFB4F84C3010
:1017800023F00203A4F84C30A663E66326647BE7EB
:1017900094F84630012B7FF461AFB4F84C3043F03D
:1017A0000203EFE794F84920616894F848304D68E7
:1017B00094F8471043EA0223204694F84620A847AD
:1017C00000283FF44BAF4368A3630368E363DDE79E
:1017D00094F84F2094F846309A42AFD02378042BE7
:1017E00010D1202383F311882046FFF7ABFE86F348
:1017F0001188636884F84F601B68032121700BB166
:101800002046984794F84630002B97D084F84F3004
:101810000423237063681B68002B8FD002212046AD
:1018200098478BE72E4BA3630223E363002388E7EB
:1018300094F8481011F0800F204601F00F010ED0EF
:1018400000F074FB012806D002287FF407AF254B77
:10185000A363E0639AE7244BA363E56396E700F094
:1018600057FBEFE700F0C4FD68E794F84630002B23
:101870007FF4F4AE94F8483013F00F013FF45EAFFC
:101880001B06204602D500F0A9FD57E700F09CFD9D
:1018900054E7032284F8342083F311882B462A4628
:1018A00029462046FFF75CFE85F3118870BD5DB1C7
:1018B000042284F8342083F311880021E36BA26BA7
:1018C0002046FFF74DFEFFE6052284F8342083F31F
:1018D00011882B462A4629462046FFF753FEE3E7A8
:1018E00004330008FC3200080033000838B590F8D3
:1018F00034300446062B22D8DFE803F037042237C1
:101900003732370090F84B1090F84A20C36B42EA08
:1019100001229A4214D9C268128AB3FBF2F502FB83
:1019200015356DB9202383F311882B462A462946A5
:10193000FFF728FE85F31188022384F8343038BD80
:10194000032384F83430202383F3118800231A46BC
:1019500019462046FFF704FE002383F3118838BDA3
:10196000036C03B198470023E7E7002100F036FD40
:101970000021204600F028FD63681B6813B1062192
:10198000204698470623D8E790F83420062A38B531
:10199000044621D80123934013F0670F1DD113F0A3
:1019A00008050FD1DB0617D5052380F83430202336
:1019B00083F311882B462A462946FFF7E3FD85F37A
:1019C000118838BDC3689B695B682BB9036C03B190
:1019D0009847002384F8343038BD002100F0FEFC25
:1019E0000021204600F0F0FC63681B6813B106215B
:1019F000204698470623EDE7836D30B500229D68A9
:101A0000446D11464FF0FF3004EB42130132954212
:101A1000C3F80019C3F81019C3F80809C3F8001B6C
:101A2000C3F8101BC3F8080BEED24FF00113C4F833
:101A30001C3830BD890141F02001016103699B061A
:101A4000FCD4122001F01AB82DE9F04F202387B002
:101A50000446456D83F3118800F1640305934FF04C
:101A6000000B2378012B04D0236E4BB96B69DB0686
:101A700006D4AB69059843F01003AB61FFF73CFB5C
:101A80008BF311884FF0000E4FF02009A36D9B6877
:101A90005FFA8EF083421BD2202383F31188E0E7A4
:101AA000616D0A6A02F4F013B3F5802F66D0B3F5C6
:101AB000402F0DD1C2F30A1602F00F0204EB82028E
:101AC00001F58051D3681F6A00231A469E4248D10F
:101AD000696911F01001E3D1012303FA00F2236ECA
:101AE0001A4200F08C8089F31188AB6823F001035F
:101AF000AB60236E23EA0203236681F3118804EBB3
:101B00008003D3F80C80D8F814100B680093431CA2
:101B10001B030293430104934868009B98425FD2E1
:101B2000B8F81060676D1B1AB34228BF3346049E95
:101B3000BE19D6F81869B6B2B3EB860F62D8029E0A
:101B4000BE1903968E680196A6F1040A9C46039E70
:101B50005AF8047F3760BCF1040F3BD9ACF1040C98
:101B6000F5E713F0030F08BF0A68072B98BF3A7018
:101B700003F101039CBF120A0137A7E7C2F30A165B
:101B800002F00F0204EB820201F58051D3689B69D9
:101B90001F68D3F808805B68A7EB030C00231F467F
:101BA0009E4208D1D36899698A684B6832443344AD
:101BB0008A604B608CE713F0030F08BF0F689C45E9
:101BC00088BF88F8007003F1010384BF3F0A08F161
:101BD0000108E5E7019E1E4403448E604B609BE7CD
:101BE000012189F31188AB6843F00103AB6021B98F
:101BF000D5F834381A43C5F834288BF311880EF120
:101C0000010E43E70021ECE710B5064C2046FFF734
:101C10005FFC4FF0A04200236265034A6366A26541
:101C2000A36610BDE80D00202C33000870B50378C2
:101C3000012B86B005465BD12F4B446D984213D1E2
:101C40002E4B5A6B42F080025A635A6942F080026E
:101C50005A6100225A610E21432001F097F9284B66
:101C6000E360284BC4F8003800232B66C4F8003E1C
:101C7000C02323604FF40413A3636E6D202000F093
:101C8000FDFE012333613369DB07FCD4122000F031
:101C9000F5FE3369002BFCDA0026A6602846FFF724
:101CA000ABFE6B68C4F81068DB68C4F81468C4F84D
:101CB0001C68FBB9144BA3614FF0FF336361AB6E3B
:101CC00093B9124B009305F17003019305F5367338
:101CD00002930223039368460D4B04930595FFF787
:101CE000D9F9A866FFF7A6F9A36843F00103A3603A
:101CF00006B070BD074BDEE7E80D0020003802405B
:101D00004014004003002002003C30C0383300087B
:101D1000491A0008083C30C0F8B5446D054600215A
:101D20002046FFF787FEA96D00234FF001128F6850
:101D3000C4F834384FF00066C4F81C284FF0FF3068
:101D400004EB431201339F42C2F80069C2F8006BF2
:101D5000C2F80809C2F8080BF2D20B68EB6563629F
:101D60006B6D10221A611E6916F01006FBD112204D
:101D700000F084FED4F8003823F4FE63C4F8003881
:101D8000A36943F4402343F01003A3610923C4F87B
:101D90001038C4F81438094BEB60094BC4F8106BC9
:101DA000C4F8003BC4F81069C4F80039EB6D03F1C6
:101DB000100243F48013EA65A362F8BD08330008FB
:101DC00040800010426D90F84E10D2F8003823F495
:101DD000FE6343EA0113C2F8003870472DE9F04171
:101DE0000EB200EB86080D46D8F80C100F6807F00D
:101DF0000303022B50D0032B50D03D4A3D4F012B03
:101E000018BF1746446D4FEA451E04EB0E0300222F
:101E1000C3F8102B8A6905F1100C002A40D04A8AB9
:101E200005F158035B013A43E2500123D4F81C2822
:101E300003FA0CF31343A6444A69C4F81C38002380
:101E4000CEF8103905F13F03002A39D00A8A898B70
:101E50009208012988BF4A43C16D04EB83035618D9
:101E600041EA0242C66529465A602046FFF7E2FD74
:101E7000D8F80C301B8A43EA85531F4305F1480309
:101E80005B01E7500123D4F81C2803FA05F515433C
:101E9000C4F81C58BDE8F081174FB3E7174FB1E7FE
:101EA00004EB4613D3F8002B22F40042C3F8002BB6
:101EB000D4F81C28012303FA0CF322EA0303BAE73F
:101EC00004EB83030E4A5A6004EB4616294620466B
:101ED000FFF7B0FDD6F8003923F40043C6F8003907
:101EE000D4F81C38012202FA05F523EA0505CFE7EC
:101EF00000800010008004100080081000800C108A
:101F000000040002826D1268C265FFF775BD000013
:101F10005831436D49015B5813F4004004D013F469
:101F2000001F14BF01200220704700004831436D9C
:101F300049015B5813F4004004D013F4001F14BF90
:101F4000012002207047000000EB8101CB68196A74
:101F50000B6813604B6853607047000000EB81030F
:101F600030B5DD68AA691368D36019B9402B84BF06
:101F7000402313606B8A1468426D1C44013CB4FB1F
:101F8000F3F46343033323F0030302EB411043EA0A
:101F9000C44343F0C043C0F8103B2B6803F0030375
:101FA000012B09B20ED1D2F8083802EB411013F41C
:101FB000807FD0F8003B14BF43F0805343F00053C0
:101FC000C0F8003B02EB4112D2F8003B43F004435F
:101FD000C2F8003B30BD00002DE9F041264D6E6D8A
:101FE00006EB40130446D3F8087BC3F8087B380798
:101FF0000AD5D6F81438190706D505EB840321460F
:10200000DB6828465B689847FA0733D5D6F814385A
:10201000DB072FD514B995F834305BB305EB840397
:10202000D968CCB98B69488A5E68B6FBF0F200FBD0
:1020300012628AB91868DA6890420DD2121A83E8DF
:102040001400202383F311880B482146FFF786FFF5
:1020500084F31188BDE8F081012303FA04F26B894F
:1020600023EA02036B81CB6823B121460248BDE815
:10207000F0411847BDE8F081E80D002000EB810336
:1020800070B5DD68436D6C692668E6604A0156BB31
:102090001A444FF40020C2F810092A6802F0030223
:1020A000012A0AB20ED1D3F8080803EB421410F447
:1020B000807FD4F8000914BF40F0805040F00050F9
:1020C000C4F8000903EB4212D2F8000940F00440C2
:1020D000C2F80009D3F83408012202FA01F10143E1
:1020E000C3F8341870BD19B9402E84BF4020206059
:1020F00020682E8A841940F00050013C1A44B4FB39
:10210000F6F440EAC440C6E72DE9F041284C666D7C
:1021100006EB40130546D3F80879C3F80879F907A8
:102120001AD5D6F81038DA0716D504EB8003D9682B
:102130004B691868DA6890422CD2121A4FF00008E6
:102140001A60C3F80480202383F3118829462046AF
:10215000FFF794FF88F311883B0619D5D6F8342889
:10216000012303FA05F5154212D0202383F31188C9
:10217000236E10482B432366D6F8343823EA05052E
:10218000C6F834580021FEF7C5FF002383F31188F9
:10219000BDE8F081012303FA05F2238923EA020353
:1021A00023818B68002BD7D0294620469847D3E758
:1021B000E80D00204C0E00202DE9F74F8048446DBB
:1021C0006669A3691E4016F4805F6661054608D003
:1021D00000230366FFF7E8F903B0BDE8F04F00F015
:1021E000A1BC002E12DAD4F8003E75489F071EBF2E
:1021F000D4F8003E23F00303C4F8003ED4F80438BA
:1022000043F00103C4F80438FFF7F8F9300504D5AA
:1022100000236B482B66FFF7E5F9B1040CD5D4F821
:10222000083813F0060FE36823F470530CBF43F42F
:10223000105343F4A053E360320704D56B68DB68A6
:102240000BB15F489847F3024ED4B7020CD5D5F8CE
:102250005480DFF86CA100274FF00109AB6D9B683B
:10226000F9B28B4280F08F80F5060DD5202383F3E1
:102270001188A369534823F01003A3610021FEF7DE
:1022800049FF002383F311883003D4F8184813D58D
:10229000E10302D50020FFF79FFEA20302D5012033
:1022A000FFF79AFE630302D50220FFF795FE27038E
:1022B00002D50320FFF790FE75038DD5E00702D508
:1022C0000020FFF721FFA10702D50120FFF71CFF27
:1022D000620702D50220FFF717FF23077FF57CAFC7
:1022E0000320FFF711FF77E7D5F854A0DFF8D4B04B
:1022F0004FF00009AB6D9B685FFA89F7BB42A4D32E
:102300000AEB4713D3F8002902F44022B2F5802FDC
:1023100036D1D3F80029002A32DAD3F8002942F066
:102320009042C3F80029D3F80029002AFBDB394684
:10233000686DFFF77FFB01232A89BB406FEA030822
:1023400008EA02022A8105EB8702D268926822B16C
:1023500039461B4801939047019B202282F3118844
:10236000DAF8342808EA0202CAF834282A6E002172
:10237000134358462B66FEF7CDFE002383F31188E6
:1023800009F10109B6E708EB4112D2F8003B03F46A
:102390004023B3F5802F10D1D2F8003B002B0CDA8C
:1023A0006A8909FA01F322EA03036B8105EB8103D1
:1023B000DB68DB680BB15046984701374EE700BF3A
:1023C000E80D00204C0E0020436D03EB4111D1F8C5
:1023D000003B43F40013C1F8003B7047436D03EB2F
:1023E0004111D1F8003943F40013C1F800397047A6
:1023F000436D03EB4111D1F8003B23F40013C1F806
:10240000003B7047436D03EB4111D1F8003923F4D1
:102410000013C1F8003970474FF0804310B51A69B6
:10242000920708D500241C61202383F3118800F053
:10243000EBFA84F31188BDE8104000F073BB000094
:102440000E4A136C43F0010313640D4A936843F082
:10245000010393604FF0804353229A624FF0FF32A2
:10246000DA6200229A615A63DA605A6001225A6184
:1024700008211A601C2000F089BD00BF003802400E
:10248000002004E000207047FEE7000070470000D5
:102490004FF0FF307047000000F0BCBD08B500F001
:1024A0006FFB00F071FABDE8084000F0FDB80000D5
:1024B00070470000022906D0032906D001290648EA
:1024C00018BF0020704705487047032A9ABF044888
:1024D00000EBC2000020704730350008E4340008EB
:1024E0000808002070B5044608460D46FEF78AFB32
:1024F000C6B22046013403780BB9184670BD324687
:102500002946FEF767FB0028F3D1012070BD0000CB
:102510002DE9F04F81469BB008460C461646FEF763
:1025200071FB3C49C5B22046FFF7DCFF08B102351C
:10253000EDB239492046FFF7D5FF08B11035EDB2AD
:10254000632D01AF0CD8DFF8DCA0DFF8DCB03D462E
:1025500094F80080B8F1000F1CD185F8008003E0EA
:102560002146384600F02AFE3846FEF74BFBC0B243
:10257000431C5B0089E84800337003237370002319
:1025800002361946DAB2904206F102063AD81BB07A
:10259000BDE8F08FB8F1250F2FD107221D49204645
:1025A000FEF718FB58B9DBF800202A60DBF804209E
:1025B0006A609BF808202A7207340935C8E70822A8
:1025C00015492046FEF706FBB8B91448AA1C10F8B6
:1025D000011F134B4FEA111E01F00F011EF80AE014
:1025E00011F80A1002F802EC984202F8011C02F1FC
:1025F0000202ECD118350834AAE785F800800134CE
:102600000135A5E7FA5C06F8022C06F8011C013337
:10261000B8E700BF90340008983400080F7AFF1F15
:102620001B7AFF1FAB340008A134000808B5202333
:1026300083F311880348FEF7B9FE002383F3118862
:1026400008BD00BFD810002010B50446052916D8D3
:10265000DFE801F016150316161D202383F31188F9
:102660000E4A0121FEF754FF20460D4A0221FEF7D3
:102670004FFF0C48FEF760FE002383F3118810BD66
:10268000202383F311880748FEF732FEF4E7202366
:1026900083F311880348FEF743FEEDE7403400085A
:1026A00064340008D810002038B50C4D0C4C0D498E
:1026B0002A4604F10800FFF72BFF05F1CA0204F1D6
:1026C00010000949FFF724FF05F5CA7204F118004C
:1026D0000649BDE83840FFF71BBF00BF9815002032
:1026E00008080020BC340008C634000898340008EC
:1026F000BFF34F8F024AD368DB03FCD4704700BF9F
:10270000003C024008B5094B1B7873B9FFF7F0FF96
:10271000074B1A69002ABFBF064A5A6002F1883285
:102720005A601A6822F480621A6008BDF617002009
:10273000003C02402301674508B50B4B1B7893B959
:10274000FFF7D6FF094B1A6942F000421A611A6876
:1027500042F480521A601A6822F480521A601A6891
:1027600042F480621A6008BDF6170020003C024067
:102770000B2870B513D80B4A0B4C137863B90B4E6A
:102780004FF0006144F8231056F8235001330C2B0E
:102790002944F7D10123137054F8200070BD0020A4
:1027A00070BD00BF28180020F81700205035000821
:1027B000014B53F820007047503500080C2070473B
:1027C0000B2810B5044601D9002010BDFFF7D0FF3B
:1027D000064B53F824301844C21A0BB9012010BD1F
:1027E00012680132F0D1043BF6E700BF5035000813
:1027F0000B2808B51BD8FFF77BFFFFF783FF0D49B8
:10280000F323CB60FFF774FFC300DBB243F4007324
:1028100043F002030B610B6943F480330B61FFF754
:1028200067FFFFF789FFBDE80840FFF7C9BF002039
:1028300008BD00BF003C02402DE9F047D407154613
:102840004DD41318B3F1016F49D2324B1B68DA072C
:1028500045D5314CFFF756FFF323E360FFF748FF00
:102860002F46401A40F20129032F884601EB00064B
:1028700018D8294C40F201197B1A4344012B01EB73
:10288000000623692FD823F001032361FFF754FFCB
:102890002846BDE8F087366851F8043CB34218D1A9
:1028A000043FE1E7B307E4D1236923F440732361D4
:1028B000236943EA090323610431D8F80030336007
:1028C000BFF34F8FFFF714FFE368002BE3D0F32330
:1028D000E360236923F001032361FFF72DFF4FF02D
:1028E000FF30BDE8F08723F440732361236943EA96
:1028F000090323618A4631F8023B3380BFF34F8FCF
:10290000FFF7F6FE3688BAF80030B6B2B342B3D05D
:10291000DFE700BF00380240003C0240084908B52C
:102920000B7828B153B9FFF7EDFE01230B7008BDFA
:1029300023B1BDE808400870FFF7FEBE08BD00BF28
:10294000F6170020014B186D704700BF00280040AB
:10295000094B1A6F120407D41A6F42F400721A67F7
:102960001A6F42F400421A67044A136843F48073F2
:102970001360034B18657047003802400070004038
:1029800000280040FEE7000010B5184CFEF7A4FA3E
:10299000FEF71EFA00F0A4F8802215492046FEF743
:1029A00053FB012344F8180C0374124B124AD968E4
:1029B00021F4E0610904090C0A431049DA60CA688D
:1029C00042F08072CA600E490A6842F001020A6051
:1029D0001022DA77202283F82220002383F3118843
:1029E00062B60848BDE81040FEF75CBBC80D002089
:1029F0008035000800ED00E00003FA05F0ED00E08E
:102A0000001000E0883500082DE9F8431A4C4FF01B
:102A1000804300256769586A04F114082E46226A2B
:102A2000BB68811A8B420CD96169414522D013449D
:102A30001B1A022B2CBFC0180230BDE8F843FEF76A
:102A400041BD134423623B68D7F80C90C3F804805F
:102A500043456361FD6001D1FEF72EFD86F31188C9
:102A60003869C847202383F311884FF08043676992
:102A7000586AD4E7BDE8F883A00D0020034B5968DD
:102A80005A68521A9042FBD8704700BF001000E00D
:102A900083691943037C81610A2B03D1436919427D
:102AA00005D170470B2B06D143698B4303D100231B
:102AB0004361FEF719BA704770B5046805460E46C3
:102AC000AC4200D170BDE3683343E36016B12269C4
:102AD000134203D0A1686068FFF7DAFF2468EFE7CC
:102AE000034B044A1A60044B044A1A60704700BF43
:102AF0002C1A0020301A0020281A00200000022082
:102B000080B5074A536823F0010300AF5360EFF329
:102B10000983683383F30988002383F3118880BD18
:102B200030EF00E098B5202300AF83F31188104BFD
:102B30005B6813F4006318D0F1EE103AEFF30984E8
:102B40004FF0807344F84C3C0A4BDB6844F8083C77
:102B5000A4F1680383F30988FEF74CFA18B1064B19
:102B600044F8503C98BD054BFAE783F3118898BDB3
:102B700000ED00E030EF00E021030008240300082E
:102B800008B500F019FA064800F0CAFAFEF79EFCF4
:102B9000FEF766FBFFF78CFCBDE80840FEF782BC41
:102BA0004433000830B5039C0172043304FB032551
:102BB000C361049B03630021059B00604060C1600A
:102BC000426102618561046242628162C162436363
:102BD00030BD00000022416A41610161C260826231
:102BE000C2626FF00101FEF7BBBA000003694269DF
:102BF000934203D1C2680AB100207047181D704784
:102C000003691960C2680132C260C26913448269F3
:102C10000361934224BF436A03610021FEF794BA23
:102C200038B504460D46E3683BB16269131D12686E
:102C3000A3621344E362002038BD237A33B92946E6
:102C40002046FEF771FA0028EDDA38BD6FF001007A
:102C5000FBE70000C368C269013BC36043691344DA
:102C600082694361934224BF436A436100238362C4
:102C7000036B03B11847704770B52023044683F3F4
:102C80001188866A3EB9FFF7CBFF054618B186F377
:102C90001188284670BDA36AE26A13F8015BA3623B
:102CA000934202D32046FFF7D5FF002383F3118818
:102CB000EFE700002DE9F74F1F4604460E46914608
:102CC000202383F311884FF080480025D8F8243062
:102CD000FB18009307F1FF3AAB46A36AABB91AF1B0
:102CE000030F06D939462046FFF79AFF68B1002343
:102CF00005E0D8F82410009A511A8F42F3D283F3DA
:102D00001188284603B0BDE8F08FA16AE36AA9EBF9
:102D100005025B1A934228BF1346402B1CD9334649
:102D200001F1400251F8040B43F8040B9142F9D130
:102D3000A36A40334036A3624035A26AE36A9A42EE
:102D400002D32046FFF786FF8BF311884D45D8D27A
:102D5000202383F31188C0E71A4630460193FDF71C
:102D60002FFF019BA26A1A441E44A2621D44E4E79D
:102D700010B5029C0172043303FB0421C3610023DC
:102D80008362C362039B0363049B00604060C46072
:102D900042610261816104624262436310BD0000CE
:102DA000026AC260426A4261026100228262C262B9
:102DB0006FF00101FEF7D4B9436902699A4203D169
:102DC000C2680AB100207047184650F8043B0B60F7
:102DD00070470000C368C2690133C360436913448C
:102DE00082694361934224BF436A43610021FEF735
:102DF000ABB9000038B504460D46E3683BB1236922
:102E00001A1DA262E2691344E362002038BD237AEE
:102E100033B929462046FEF787F90028EDDA38BD98
:102E20006FF00100FBE7000003691960C268013A16
:102E3000C260C269134482690361934224BF436A3A
:102E4000036100238362036B03B1184770470000DE
:102E500070B5202304460E4683F31188856A35B980
:102E60001146FFF7C7FF10B185F3118870BDA36A43
:102E70001E70A36AE26A01339342A36204D3E1693C
:102E800020460439FFF7D0FF002080F3118870BD81
:102E90002DE9F74F1F4604460D469146202383F344
:102EA00011884FF080480026D8F82430FB18009392
:102EB00007F1FF3AB346A36AABB91AF1030F06D97B
:102EC00039462046FFF796FF68B1002305E0D8F8A1
:102ED0002410009A511A8F42F3D283F3118830469E
:102EE00003B0BDE8F08FA06AE36AA9EB06021B1AE3
:102EF000934228BF1346402B1CD905F1400355F8D7
:102F0000042B40F8042B9D42F9D1A36A4033A362FD
:102F10004036A26AE36A9A4204D3E1692046043942
:102F2000FFF782FF8BF311884E45D8D2202383F31D
:102F30001188C0E71A4629460193FDF741FE019B1F
:102F4000A26A1A441D44A2621E44E2E70269436970
:102F50009A4203D1C3681BB9184670470023FBE7A8
:102F6000836A002BF8D0043B9B1AF5D01360C3682A
:102F7000013BC360C3691A44836902619A4224BF5A
:102F8000436A0361002383620123E5E700F16043A4
:102F900000F01F02400903F5614309018000C9B236
:102FA00000F1604083F8001300F561400123934075
:102FB000C0F8803103607047144B00211A694FF04C
:102FC000FF321A61196158695A615961186A60F0D3
:102FD000805018621962586A5A6259621A6C42F03B
:102FE00080521A640A4A106840F480701060186FAA
:102FF00000F44070B0F5007F1EBF4FF480301867BA
:103000001967536823F40073536070470038024017
:1030100000700040314B4FF080521A64304A4FF438
:10302000404111601A6842F001021A601A68920762
:10303000FCD59A6822F003029A609A689A60274B3E
:1030400019469A6812F00C02FBD1186800F0F900DA
:1030500018609A601A6842F480321A600B689B0309
:10306000FCD54B6F43F001034B671C4B5A6F900725
:10307000FCD51C4A5A601A6842F080721A60184ADD
:1030800053685904FCD5154B1A689201FCD5164AB1
:103090009A60164B1A68164B9A42164B1AD1164A6A
:1030A0001168164A914215D140F205121A600B4B75
:1030B0009A6842F002029A609A6802F00C02082AAA
:1030C000FAD15A6C42F480425A645A6E42F48042F9
:1030D0005A66704740F20572E8E700BF00380240C8
:1030E000007000400854400700948838002004E035
:1030F00011640020003C024000ED00E041C20F419D
:103100004B6843608B688360CB68C3600B69436125
:103110004B6903628B6943620B6803607047000070
:103120001C4B0246186B10B540F2FF142043186385
:10313000196D1948214319651146FFF7E1FF17483A
:1031400002F11C01FFF7DCFF154802F13801FFF71F
:10315000D7FF144802F15401FFF7D2FF124802F1E1
:103160007001FFF7CDFF114802F18C01FFF7C8FF96
:103170000F4802F1A801FFF7C3FF0E4802F1C40196
:10318000FFF7BEFF0C4802F1E001BDE81040FFF779
:10319000B7BF00BF003802400000024000040240F8
:1031A00000080240000C02400010024000140240DF
:1031B00000180240001C02400020024080EA010288
:1031C000844612F0030F4FD111F0030F32D14DF8A6
:1031D000044D11F0040F51F8043B0BD0A3F1013260
:1031E0009A4312F0803F04BF4CF8043B51F8043B73
:1031F00016D100BF51F8044BA3F101329A4312F0EB
:10320000803FA4F101320BD14CF8043BA24312F0F1
:10321000803F04BF51F8043B4CF8044BEAD02346EE
:103220000CF8013B13F0FF0F4FEA3323F8D15DF8A0
:10323000044B704711F0010F06D011F8012B0CF868
:10324000012B002A08BF704711F0020FBFD031F8E0
:10325000022B12F0FF0F16BF2CF8022B8CF8002067
:1032600012F47F4FB3D1704711F8012B0CF8012BEA
:10327000002AF9D1704700BF12101213121100007A
:1032800053544D3332463F3F3F00000000000000E2
:10329000803200083F00000013040000BC32000828
:1032A0003F00000019040000C63200083F00000083
:1032B00021040000D03200083F00000053544D3379
:1032C00032463430780053544D333246343278002D
:1032D00053544D333246343436585800DD1100080B
:1032E000C911000805120008F1110008FD110008BD
:1032F000E9110008D5110008C11100080000000004
:10330000010000000000000000000000111600088D
:10331000ED1800088919000840004000C010002086
:10332000C010002001000000D0100020800000002C
:1033300040010000030000007573625F70756D70DE
:10334000000000000000801200000000AAAAAAAA43
:1033500000000000FFBF00000000000000A00A0005
:103360000000040000000000AAAAAAAA00000000B1
:10337000FFFD000000000000000000000000000051
:1033800000000000AAAAAAAA00000000FFFF000097
:10339000000000000000000000000000000000002D
:1033A000AAAAAAAA00000000FFFF00000000000077
:1033B000000000000000000000000000AAAAAAAA65
:1033C00000000000FFFF00000000000000000000FF
:1033D0000000000000000000AAAAAAAA0000000045
:1033E000FFFF0000000000000000000000000000DF
:1033F00000000000AAAAAAAA00000000FFFF000027
:1034000000000000000000000000000000000000BC
:103410000A0000000000000003000000000000009F
:10342000000000000000000000000000000000009C
:10343000000000000000000000000000000000008C
:103440000200000000000000F913000861140008E9
:1034500040004000681500207815002002000000A0
:10346000000000000300000000000000A11400089C
:10347000000000001000000088150020000000007F
:103480000100000000000000E80D00200101020022
:1034900025424F41524425002553455249414C2570
:1034A000004D6174656B4634303500303132333451
:1034B00035363738394142434445460041726475D8
:1034C00050696C6F740025424F415244252D424C87
:1034D0000000000049260008B52400086513000814
:1034E0002D26000843000000EC34000809024300C8
:1034F000020100C03209040000010202010005249B
:103500000010010524010001042402020524060024
:1035100001070582030800FF09040100020A0000F8
:10352000000705010240000007058102400000007D
:10353000120000003835000812011001020000409E
:103540008304405700020102030100000403090440
:10355000004000000040000000400000004000006B
:103560000000010000000200000002000000020054
:103570000000020000000200000002000000020043
:103580006D61696E00000000A03500083018002051
:10359000281A002001000000852900080000000012
:1035A00069646C6500000000FF00960000000008E0
:1035B000040000004C35000800000000000000007E
:1035C00000000000000000000000000000000000FB
:00000001FF
